:10000000A72800380319A228A80020088400211876
:100010008317A001A101A81B15280008A000A81C97
:10002000A228840A0008A100A2281A200005031DA6
:10003000A00AA22800308A00280807398207013464
:10004000023404340834103420344034803421081D
:1000500020040319A00A8030201AA1062019A10645
:10006000A018A106210DA00DA10DA228A301A20098
:10007000FF30A207031CA307031CA2280330A10022
:10008000DF3044203828A101E83EA000A109FC305F
:10009000031C4D28A00703184A28A0076400A10FDD
:1000A0004A2820185328A01C572800005728080069
:1000B000A20001306028A20004306028A2000530B0
:1000C000A80023082102031D67282208200204300B
:1000D00003180130031902302805031DFF30A22840
:1000E000A501A4011030A600210DA40DA50D220824
:1000F000A4022308031C230FA50203188628220844
:10010000A40723080318230FA5070310A00DA10DB2
:10011000A60B74282008A2281030A800A101A00175
:10012000A70CA60C031C9A282208A0072308031872
:10013000230FA107A10CA00CA50CA40CA80B9028C0
:100140002408A22883130313831264000800831673
:10015000870185018312CC01CD014C08A0004D0818
:10016000A100A3010D308A0158208A11031DFD2B27
:100170004D088A11031D28294C08A2000C3C8A1145
:10018000031C28290310220DA2078A11D720A000E2
:10019000A20A8A11D720A100A20A8A11D7208A01B7
:1001A00001202008CE002108CF008A112829013023
:0601B0008A00220800296C
:1002000082070134003400340A34003400340234EC
:10021000003400340B34003400340934003400342A
:100220000334003400340C34003400340834003417
:1002300000340434003400340D3400340034073406
:100240000034003405340034003406340034003403
:100250004E08A0004F08A100A30101308A015E20D2
:100260008A11031D4E290130D000D1015008A00091
:100270005108A100A30103308A0158208A11031DEF
:100280004C294B30F400F5018A11FF23D00A0319E1
:10029000D10A8A11031D36298A11F72B4E08A000B6
:1002A0004F08A100A30102308A015E208A11031DBC
:1002B00078290130D200D3015208A0005308A100D0
:1002C000A30102308A0158208A11031D7629643067
:1002D000EA00EB015E30E4000130E5008A11AE2750
:1002E000D20A0319D30A8A11031D5C298A11F72B3C
:1002F0004E08A0004F08A100A30103308A015E2030
:100300008A11031DDF291330F0000130F10070085D
:10031000A0007108A100A30196308A015B208A1118
:10032000031DA2298A1193271930F00200308A1187
:1003300003189E29013E8A110318A229F1028A118D
:10034000031887299630F000F1017008A0007108A9
:10035000A100A3014B308A015B208A11031DC02933
:100360008A1193270530F00200308A110318BC2946
:10037000013E8A110318C029F1028A110318A52928
:100380000130D400D5015408A0005508A100A301F4
:1003900007308A0158208A11031DD6298A11932714
:1003A000D40A0319D50A8A11031DC32985018701BF
:1003B0007108A30070088A0137208A11F72B4E08B4
:1003C000A0004F08A100A30104308A015E208A1119
:1003D000031D462A1330F2000130F3007208A0001A
:1003E0007308A100A30196308A015B208A11031DC6
:1003F000092A8A1180271930F20200308A11031865
:10040000052A013E8A110318092AF3028A110318EA
:10041000EE299630F200F3017208A0007308A100E3
:10042000A3014B308A015B208A11031D272A8A1100
:1004300080270530F20200308A110318232A013E7A
:100440008A110318272AF3028A1103180C2A013093
:10045000D600D7015608A0005708A100A301073015
:100460008A0158208A11031D3D2A8A118027D60A45
:100470000319D70A8A11031D2A2A850187017308E7
:10048000A30072088A0137208A11F72B4E08A000BA
:100490004F08A100A30105308A015E208A11031DC7
:1004A0006C2A0130D800D9015808A0005908A100D1
:1004B000A30104308A0158208A11031D6A2A4B3097
:1004C000DA00DB018A117F26D80A0319D90A8A11BA
:1004D000031D542A8A11F72B4E08A0004F08A100D3
:1004E000A30106308A015E208A11031D922A013081
:1004F000BA00BB013A08A0003B08A100A3010430E8
:100500008A0158208A11031D902AC830F600F7018D
:100510008A113626BA0A0319BB0A8A11031D7A2AE0
:100520008A11F72B4E08A0004F08A100A301073045
:100530008A015E208A11031DB82A0130BC00BD016A
:100540003C08A0003D08A100A30104308A01582006
:100550008A11031DB62AC830E000E1018A11F32593
:10056000BC0A0319BD0A8A11031DA02A8A11F72BA0
:100570004E08A0004F08A100A30108308A015E20A8
:100580008A11031DDE2A0130BE00BF013E08A00013
:100590003F08A100A30104308A0158208A11031DDD
:1005A000DC2AC830DE00DF018A11D025BE0A03191B
:1005B000BF0A8A11031DC62A8A11F72B4E08A00014
:1005C0004F08A100A30109308A015E208A11031D92
:1005D000042B0130C000C1014008A0004108A10067
:1005E000A30103308A0158208A11031D022BC83051
:1005F000E200E3018A112B25C00A0319C10A8A11FE
:10060000031DEC2A8A11F72B4E08A0004F08A10009
:10061000A3010A308A015E208A11031D272B0130B5
:10062000C200C3014208A0004308A100A301143086
:100630008A0158208A11031D252B8A11AA24C20A77
:100640000319C30A8A11031D122B8A11F72B4E08B6
:10065000A0004F08A100A3010B308A015E208A117F
:10066000031D4D2B6430E800E9010130C400C501D1
:100670004408A0004508A100A30104308A015820C5
:100680008A11031D4B2B8A150F20C40A0319C50AB2
:100690008A11031D382B8A11F72B4E08A0004F0832
:1006A000A100A3010C308A015E208A11031DD62B04
:1006B0000130C600C7014608A0004708A100A301F9
:1006C00003308A0158208A11031DD42B8316200879
:1006D0008312A000831621088312A1008A0127201B
:1006E00020088316A000831221088316A100200889
:1006F0008312A000831621088312A1001030A200EB
:100700000430A3008A0170208316A20083122108FE
:100710008316A30083120530A600A70183162208C2
:100720008312A200831623088312A3008A018C205F
:10073000DC002508DD0064305C078316A40083120A
:100740005D080318013E8316A50022088312A0004D
:10075000831623088312A1000930A200A3018A0195
:1007600070208316A600831221088316A700831227
:100770000530A600A701831622088312A200831663
:1007800023088312A3008A018C208316A8008312F9
:1007900025088316A90083128A158E20C60A03191C
:1007A000C70A8A11031D5B2B8A11F72B4E08A00084
:1007B0004F08A100A3010D308A015E208A11031D9C
:1007C000F72B0130C800C9014808A0004908A10062
:1007D000A30104308A0158208A11031DF72B8A15C2
:1007E0000421C80A0319C90A8A11031DE42BCC0A83
:1007F0000319CD0A8A11031DAD288A01AB280130E7
:10080000870085017508A30074088A0137200B3022
:10081000870085017508A30074088A0137201F30FE
:100820008700013085007508A30074088A0137200D
:100830003F308700033085007508A30074088A01E3
:1008400037203F308700073085007508A300740803
:100850008A0137203E308700073085007508A300E5
:1008600074088A0137203430870007308500750806
:10087000A30074088A0137202030870006308500E5
:100880007508A30074088A013720870104308500A9
:100890007508A30074088A0137208701850175084F
:1008A000A30074088A013720043087008501750889
:1008B000A30074088A013720263087008501750857
:1008C000A30074088A013720373087000430850080
:1008D0007508A30074088A0137203F30870006306E
:1008E00085007508A30074088A0137203F3087000F
:1008F000073085007508A30074088A0137203B3053
:100900008700073085007508A30074088A01372026
:1009100019308700073085007508A30074088A0124
:10092000372008308700033085007508A30074085D
:100930008A0137208701013085007508A3007408FB
:100940008A013720870185017508A30074088A0190
:1009500037200800831620088312A0008316210880
:100960008312A1008A01272020088316A000831289
:1009700021088316A10020088312A00083162108F5
:100980008312A1001030A2000430A3008A0170205D
:100990008316A200831221088316A30083120A3053
:1009A000A600A701831622088312A200831623083B
:1009B0008312A3008A018C20DC002508DD0064304E
:1009C0005C078316A40083125D080318013E83169A
:1009D000A50022088312A000831623088312A10019
:1009E0000930A200A3018A0170208316A600831299
:1009F00021088316A70083120A30A600A7018316D8
:100A000022088312A200831623088312A3008A01FE
:100A10008C208316A800831225088316A9002608B7
:100A20008312850083162208831287008316250807
:100A30008312A3008316240883128A0137208501BC
:100A40008701831629088312A300831628088312BE
:100A50008A01372008000830870085016308A30059
:100A600062088A0137201130870001308500630851
:100A7000A30062088A0137202230870002308500F7
:100A80006308A30062088A0137200430870004301D
:100A900085006308A30062088A0137208701850169
:100AA0006308A30062088A013720023087008501AD
:100AB0006308A30062088A0137201530870085018A
:100AC0006308A30062088A013720283087000230BB
:100AD00085006308A30062088A013720870105307A
:100AE00085006308A30062088A0137208701850119
:100AF0006308A30062088A0137202030870085013F
:100B00006308A30062088A0137201430870004308C
:100B100085006308A30062088A0137200A30870035
:100B2000023085006308A30062088A013720013083
:100B30008700013085006308A30062088A0137201E
:100B4000870185016308A30062088A0137208701B5
:100B5000023085006308A30062088A013720103044
:100B60008700053085006308A30062088A013720EA
:100B70002A30870085016308A30062088A013720B4
:100B80000530870085016308A30062088A013720C9
:100B9000870185016308A30062088A0137200800E5
:100BA00020308700063085005F08A3005E088A01B8
:100BB00037200B30870085015F08A3005E088A019B
:100BC00037202630870085015F08A3005E088A0170
:100BD000372008308700033085005F08A3005E08D7
:100BE0008A01372008000430870085016108A300CE
:100BF00060088A01372009308700013085006108CC
:100C0000A30060088A01372087010430850061084D
:100C1000A30060088A01372007308700850161083A
:100C2000A30060088A013720870101308500610830
:100C3000A30060088A013720243087000430850033
:100C40006108A30060088A01372001308700850110
:100C50006108A30060088A013720870107308500FA
:100C60006108A30060088A01372008001730870058
:100C7000023085007708A30076088A0137203630D5
:100C80008700013085007708A30076088A013720A5
:100C90003C308700043085007708A30076088A017D
:100CA000372031308700063085007708A3007608AA
:100CB0008A01372012308700073085007708A300AB
:100CC00076088A0137201C308700033085007708BA
:100CD000A30076088A01372039308700013085006B
:100CE0007708A30076088A0137201B30870004307C
:100CF00085007708A30076088A01372008000430B1
:100D0000870085015B08A3005A088A01372002305A
:100D1000870085015B08A3005A088A01372001304B
:100D2000870085015B08A3005A088A013720083034
:100D3000870085015B08A3005A088A01372010301C
:100D4000870085015B08A3005A088A0137202030FC
:100D5000870085015B08A3005A088A013720043008
:100D6000850087015B08A3005A088A0137200230FA
:100D7000850087015B08A3005A088A0137200130EB
:100D8000850087015B08A3005A088A0137200830D4
:100D9000870085015B08A3005A088A0137201030BC
:100DA000870085015B08A3005A088A0137200230BA
:100DB000850087015B08A3005A088A0137200130AB
:100DC000850087015B08A3005A088A013720083094
:100DD000870085015B08A3005A088A01372001308B
:100DE000870085015B08A3005A088A01372002307A
:100DF000870085015B08A3005A088A01372010305C
:100E0000870085015B08A3005A088A01372020303B
:100E1000870085015B08A3005A088A013720043047
:100E2000870085015B08A3005A088A013720023039
:100E3000870085015B08A3005A088A01372001302A
:100E4000870085015B08A3005A088A013720083013
:100E5000870085015B08A3005A088A01372001300A
:100E6000850087015B08A3005A088A0137200230F9
:100E7000850087015B08A3005A088A0137200430E7
:100E8000850087015B08A3005A088A0137202030BB
:100E9000870085015B08A3005A088A0137201030BB
:100EA000870085015B08A3005A088A0137200230B9
:100EB000850087015B08A3005A088A0137200130AA
:100EC000850087015B08A3005A088A013720083093
:100ED000870085015B08A3005A088A01372001308A
:100EE000870085015B08A3005A088A013720023079
:100EF000870085015B08A3005A088A013720080093
:100F0000850187017308A30072088A0137203F30EA
:100F10008700073085007308A30072088A01372014
:100F20008701850108001030870085017108A30042
:100F300070088A0137202A30870002308500710846
:100F4000A30070088A01372005308700053085002E
:100F50007108A30070088A01372008008701850105
:100F60006B08A3006A088A01372013308700063017
:100F700085006508A30064088A0137208701850180
:100F80006B08A3006A088A0137203D3087000530CE
:100F900085006508A30064088A0137208701850160
:100FA0006B08A3006A088A0137203D3087000230B1
:100FB00085006508A30064088A0137208701850140
:100FC0006B08A3006A088A0137203D30870005308E
:100FD00085006508A30064088A0137208701850120
:100FE0006B08A3006A088A0137203D308700023071
:100FF00085006508A30064088A0137208701850100
:101000006B08A3006A088A0137203F30870001304F
:1010100085006508A30064088A01372008000930AC
:10102000870085016908A30068088A0137202830F5
:10103000870085016908A30068088A013720083005
:101040008700023085006908A30068088A013720FC
:101050000630870085016908A30068088A013720E7
:101060001130870085016908A30068088A013720CC
:1010700002308700013085006908A30068088A01F2
:1010800037201130870085016908A30068088A01AC
:1010900037208701063085006908A30068088A01A7
:1010A000372004308700013085006908A3006808F4
:1010B0008A01372010308700013085006908A300BD
:1010C00068088A0137202230870085016908A3005B
:1010D00068088A01372010308700043085006908CD
:1010E000A30068088A01372003308700850169085A
:1010F000A30068088A013720143087008501690839
:10110000A30068088A01372020308700023085005C
:101110006908A30068088A013720080006308700A4
:1011200003308500831629088312A300831628083C
:1011300083128A013720033087000630850083162A
:1011400025088312A3008316240883128A013720FE
:101150002930870004308500831629088312A300F4
:101160008316280883128A0137202C30870001302B
:101170008500831625088312A30083162408831292
:101180008A0137200630870003308500831629083E
:101190008312A3008316280883128A0137202C307B
:1011A000870001308500831625088312A30083166B
:1011B000240883128A0137202930870004308500F3
:1011C000831629088312A3008316280883128A0134
:1011D00037200330870006308500831625088312E8
:1011E000A3008316240883128A0137200630870063
:1011F00003308500831629088312A300831628086C
:1012000083128A01372008002F30870007308500BD
:101210006308A30062088A01372010308700850127
:0C1220006308A30062088A013720080060
:02400E00FC3F75
:00000001FF
